:10000000A3C00000BCC00000BAC00000B8C000001F
:10001000B6C00000B4C00000B2C00000B0C0000014
:10002000AEC00000ACC00000AAC00000C9C3000000
:100030006AC40000A4C00000A2C00000A0C000006C
:100040009EC000009CC000009AC0000098C0000044
:1000500096C0000094C0000092C00000ACC1000037
:100060008EC000008CC000008AC0000088C0000064
:1000700086C0000084C0000082C0000080C0000074
:100080007EC000007CC000007AC0000078C0000084
:1000900076C0000074C000001201100102000008C8
:1000A000EB03602000000102DC0109023E000201B6
:1000B00000C0320904000001020201000524001002
:1000C0000104240206052406000107058203080036
:1000D000FF09040100020A000000070504021000E5
:1000E00005070583021000050403090436034400D4
:1000F0005300700061006300650020002800770055
:10010000770077002E0064007300700061006300C8
:1001100065002E006F00720067002E006E007A00EE
:1001200029000000220344005300700061006300B6
:100130006500200052006F0062006F007400200014
:1001400032002E003000000011241FBECFEFD2E09D
:10015000DEBFCDBF11E0A0E0B1E0E0E9FFE002C00A
:1001600005900D92AE31B107D9F712E0AEE1B1E0E2
:1001700001C01D92A534B107E1F76BD007C740CF8E
:10018000FC01A081B1816C93808191810196918362
:100190008083268137818217930721F4848195819A
:1001A000918380832FB7F8948285938501969387F6
:1001B00082872FBF0895FC01A281B3818D91B38303
:1001C000A28326813781A217B30721F424813581C8
:1001D000338322839FB7F8942285338521503040A2
:1001E000338722879FBF0895FC012FB7F89471834E
:1001F0006083738362837583648360587F4F7783E2
:10020000668380E890E091878087138612862FBFEF
:10021000089584B7877F84BF28E10FB6F8942093B0
:100220006000109260000FBE83E390E09093CD00D9
:100230008093CC0086E08093CA001092C80020937F
:10024000C900539A5A9AACD284E085BD5C9A549AFC
:100250000895CF93DF93DDDF8DE292E06EE171E0F0
:10026000C3DF81E292E06EE971E0BEDF78948FB780
:10027000F89420913702309138028FBF8091350277
:10028000909136022817390749F080E091E02ED688
:10029000BC0197FD03C08DE292E072DF8FB7F89446
:1002A000C0912B02D0912C028FBFA89908C08091D9
:1002B000290290912A020A978C179D0790F4A89A18
:1002C0000EC0E0912302F091240280E091E0608171
:1002D000A4D52197882329F481E292E06CDF20974E
:1002E00081F78091C80085FF0EC02FB7F8948091E8
:1002F0003702909138022FBF009729F08DE292E0EB
:100300005ADF8093CE0080E091E0E1D537D3AFCFC4
:1003100080E091E05EC580E091E0AFC41F93FC01F6
:10032000A18DA150A23028F4B0E0A55EBE4F1C9173
:1003300001C010E0808D823009F41860828D873012
:1003400031F0883031F0863029F4126003C0146037
:1003500001C016601092C9001092C8001092CA0025
:100360002489358946895789203081EE380780E015
:10037000480780E0580721F428EC35EE40E050E0D3
:10038000CA01B9019695879577956795605C7D4B15
:10039000804F9F4FD9D5215030403093CD002093CE
:1003A000CC001093CA0082E08093C80088E9809353
:1003B000C9001F9108951F920F920FB60F9211243A
:1003C0002F933F934F935F936F937F938F939F935D
:1003D000AF93BF93EF93FF936091CE008EB38430C1
:1003E00019F481E292E0CCDEFF91EF91BF91AF91E1
:1003F0009F918F917F916F915F914F913F912F913D
:100400000F900FBE0F901F901895FC01208920FFC0
:1004100002C05C9808955C9A0895923029F0933058
:1004200041F09130E9F417C02EE330E0EAEAF0E061
:100430001BC0813041F0813018F0823089F406C051
:10044000E8EEF0E005C0ECEEF0E002C0E4E2F1E03E
:10045000249130E009C022E130E0E8E9F0E004C096
:1004600020E030E0E0E0F0E0DA011196FC93EE935A
:10047000C90108958F708093E900EBEEF0E0808170
:1004800081608083EDEEF0E010826093EC004083A9
:100490008091EE00881F8827881F0895EF92FF92B1
:1004A0000F931F93CF93DF93162FE82EE7017E0162
:1004B000F92EE70100E02AC09881992329F16B8188
:1004C000E981FA812C81892F8F70853018F562952A
:1004D000660F660F607C991F9927991F692B223040
:1004E00010F096E001C092E028E030E040E003C068
:1004F0004F5F220F331F2E173F07D0F34295407FE7
:10050000492BB8DF882331F00F5F25960117A0F241
:1005100081E001C080E0DF91CF911F910F91FF90AA
:10052000EF90089580913A0287FF11C003C08EB307
:100530008823B1F08091E80082FFF9CF8091E80034
:100540008B778093E80008958EB3882349F08091DB
:10055000E80080FFF9CF8091E8008E778093E80073
:1005600008958091E4009091E50044E62091EC002C
:1005700020FF25C02091E80020FD15C02EB32223C6
:10058000A1F02530A1F02091EB0025FD12C02091B3
:10059000E4003091E5002817390741F3442359F06E
:1005A0004150C901E3CF80E0089582E0089583E0DF
:1005B000089581E0089584E0089580E008952091F1
:1005C000E80022FFDBCFF9CF282F392FF9018091E6
:1005D0004002909141028617970718F4BC0120E071
:1005E00034C061157105D9F78091E8008E7780934A
:1005F000E800F5CF8EB38823E9F18530B9F1809119
:10060000E80083FD35C08091E80082FD29C080911B
:10061000E80080FF1AC08091F20090E006C02191AE
:100620002093F1006150704001966115710519F039
:1006300088309105A0F321E08830910509F020E091
:100640008091E8008E778093E8006115710591F63E
:10065000222381F605C08EB3882361F0853061F0D6
:100660008091E80082FFF7CF80E0089583E008954D
:1006700081E0089582E0089583E00895E82FF92F3E
:1006800080914002909141028617970718F4BC01AF
:1006900020E036C061157105D9F78091E8008E77AA
:1006A0008093E800F5CF8EB3882309F43EC08530EF
:1006B000C1F18091E80083FD36C08091E80082FDA1
:1006C0002AC08091E80080FF1BC08091F20090E07A
:1006D00007C024912093F10031966150704001963B
:1006E0006115710519F08830910598F321E0883083
:1006F000910509F020E08091E8008E778093E80072
:100700006115710581F6222371F605C08EB3882329
:1007100061F0853061F08091E80082FFF7CF80E0E2
:10072000089583E0089581E0089582E0089583E0CC
:10073000089540D042D08091D8008F778093D80020
:100740008091D80080688093D8008091D8008F7DF8
:100750008093D80019BC82E089BD09B400FEFDCFAA
:100760001EBA10924202109244021092430280E09C
:1007700060E042E07FDE8091E1008E7F8093E100C7
:100780008091E20081608093E2008091E2008860C5
:100790008093E2008091E0008E7F8093E0000895D6
:1007A000E3E6F0E080818E7F808381E080933902F0
:1007B000C0CF08951092E20008951092E1000895CC
:1007C0001F920F920FB60F9211242F933F934F93C6
:1007D0005F936F937F938F939F93AF93BF93EF93A9
:1007E000FF938091E10082FF0AC08091E20082FFC6
:1007F00006C08091E1008B7F8093E100DADF809179
:10080000E10080FF16C08091E20080FF12C080915D
:10081000E2008E7F8093E2008091E200806180930D
:10082000E2008091D80080628093D80019BC1EBA83
:10083000C0DF8091E10084FF2BC08091E20084FF43
:1008400027C019BC82E089BD09B400FEFDCF8091AC
:10085000D8008F7D8093D8008091E1008F7E8093B7
:10086000E1008091E2008F7E8093E2008091E200BF
:1008700081608093E20080914202882321F480917C
:10088000E30087FF02C084E001C081E08EBB91DFFE
:100890008091E10083FF26C08091E20083FF22C0A7
:1008A0008091E100877F8093E10082E08EBB10920F
:1008B00042028091E1008E7F8093E1008091E2000E
:1008C0008E7F8093E2008091E20080618093E2005D
:1008D00080E060E042E0CEDD8091F00088608093AF
:1008E000F00067DFFF91EF91BF91AF919F918F91E2
:1008F0007F916F915F914F913F912F910F900FBE1C
:100900000F901F9018951F920F920FB60F921124FF
:100910001F932F933F934F935F936F937F938F9387
:100920009F93AF93BF93EF93FF931091E9001F70D4
:100930008091EC001092E9008091F000877F809315
:10094000F000789436D01092E9008091F000886031
:100950008093F0001093E900FF91EF91BF91AF9168
:100960009F918F917F916F915F914F913F912F91C7
:100970001F910F900FBE0F901F9018951F938EB36D
:100980008823A9F08091E9008F709091EC0090FF8E
:1009900002C010E801C010E0182B1092E90080910D
:1009A000E80083FF01C005D01F701093E9001F917C
:1009B00008950F931F93DF93CF93CDB7DEB7AC9716
:1009C0000FB6F894DEBF0FBECDBFEAE3F2E0809130
:1009D000F100819322E0E234F207C9F79CDC8091B8
:1009E000E80083FF31C180913A0220913B0225301B
:1009F00009F484C0263040F42130A1F1213070F098
:100A0000233009F021C12EC0283009F4F0C029306C
:100A100009F4FFC0263009F017C193C0803821F0D7
:100A2000823809F011C108C08091430290914402BC
:100A3000992371F082600CC080913E028F70809388
:100A4000E9009091EB0081E095FF80E01092E900D1
:100A50009091E800977F9093E8008093F1001092C6
:100A6000F100D0C0882319F0823009F0EDC090E089
:100A70008F719070009729F08230910509F0E4C0E1
:100A80000BC080913C02813009F0DEC0233009F0B8
:100A900080E0809344022CC080913C02882341F581
:100AA00020913E022F7009F4CFC02093E90080917D
:100AB000EB0080FF1DC080913B02833021F48091C8
:100AC000EB00806213C08091EB0080618093EB00AB
:100AD00081E090E002C0880F991F2A95E2F7809389
:100AE000EA001092EA008091EB0088608093EB00AE
:100AF0001092E9008091E800877F87C0882309F081
:100B0000A3C010913C021F770FB7F8948091E800C2
:100B1000877F8093E80006DD8091E80080FFFCCFAE
:100B20008091E3008078812B8093E300806880933C
:100B3000E300112311F083E001C082E08EBB0FBF00
:100B400083C08058823008F07FC080913C02909131
:100B50003D0223E08C3D920791F583E08C838AE28D
:100B60008B835FB7F894DE01159680E090E04EE04D
:100B700061E2E42FF0E060935700E49180FF03C04E
:100B8000E295EF704F5FEF702E2F30E0EA3018F0F3
:100B9000295C3F4F02C0205D3F4F2D933D9301964E
:100BA0008431910531F75FBF8091E800877F8093A2
:100BB000E800CE0103966AE270E006DD12C06091A3
:100BC0003E02AE014F5F5F4F28DCBC01009709F485
:100BD0003BC08091E800877F8093E80089819A81FB
:100BE0004DDD8091E8008B778093E8002DC0803840
:100BF00059F58091E800877F8093E8008091420258
:100C00008093F1008091E8008E778093E8008ADC81
:100C10001BC08823C9F490913C029230A8F48091C3
:100C2000E800877F8093E800909342027BDC80910C
:100C30004202882321F48091E30087FF02C084E010
:100C400001C081E08EBB64DB8091E80083FF0AC0B5
:100C50008091EB0080628093EB008091E800877FB9
:100C60008093E800AC960FB6F894DEBF0FBECDBF00
:100C7000CF91DF911F910F910895CF93DF93EC01F6
:100C80008091E80083FFA2C0888190E020913E021D
:100C900030913F022817390709F098C080913B0234
:100CA000813269F0823220F4803209F08FC03CC07A
:100CB000823209F46AC0833209F088C079C0809119
:100CC0003A02813A09F082C08091E800877F8093E0
:100CD000E8008091E80080FFFCCF8C899D89AE8977
:100CE000BF898093F100292F3A2F4B2F552720934E
:100CF000F1009D01442755272093F1008B2F992760
:100D0000AA27BB278093F100888D8093F100898DFD
:100D10008093F1008A8D8093F1008091E8008E77B6
:100D20008093E800FFDB52C080913A02813209F0E3
:100D30004DC08091E800877F8093E80004C08EB3A7
:100D4000882309F443C08091E80082FFF8CF3091F6
:100D5000F1002091F1009091F1008091F1003C8B25
:100D60002D8B9E8B8F8B8091F100888F8091F1006D
:100D7000898F8091F1008A8F8091E8008B77809332
:100D8000E800D0DBCE01CADA21C080913A0281327C
:100D9000E9F48091E800877F8093E800C3DB8091CD
:100DA0003C0290913D02998B888BCE012EDB0EC0C8
:100DB00080913A02813251F48091E800877F8093DC
:100DC000E800B0DBCE0160913C02BDD0DF91CF9155
:100DD0000895CF93DF93EC014096FC018BE0DF0197
:100DE0001D928A95E9F782E08C83898783E08E875C
:100DF000CE01019661E052DB882359F0CE010696C0
:100E000061E04CDB882329F0CE010B9661E046DBE4
:100E100001C080E0DF91CF910895DF93CF930F92CF
:100E2000CDB7DEB7FC018EB38430F9F4248935895F
:100E3000468957892115310541055105B1F0818158
:100E40008F708093E9008091E80085FD0AC0809151
:100E5000E8008E778093E800698383DB69818823CB
:100E600029F46093F10080E001C082E00F90CF91FF
:100E7000DF910895FC018EB3843019F524893589FA
:100E8000468957892115310541055105D1F08181E8
:100E90008F708093E9008091F2008823A1F09091F7
:100EA000E8008091E8008E778093E80095FD0DC002
:100EB00058DB882359F49091E8009E779093E800DE
:100EC000089582E0089580E0089580E008952EB3AB
:100ED000243059F4FC012489358946895789211524
:100EE00031054105510509F0C5CF0895FC018EB3C8
:100EF000843029F52489358946895789211531059A
:100F000041055105E1F086818F708093E900809161
:100F1000E80082FF14C08091F200882321F0209124
:100F2000F10030E002C02FEF3FEF8091F200882304
:100F300041F48091E8008B778093E80002C02FEFA6
:100F40003FEFC90108950895A1E21A2EAA1BBB1B09
:100F5000FD010DC0AA1FBB1FEE1FFF1FA217B30785
:100F6000E407F50720F0A21BB30BE40BF50B661F9B
:100F7000771F881F991F1A9469F76095709580955F
:100F800090959B01AC01BD01CF010895F894FFCF6E
:100F9000008310000001041000000182080000011D
:0E0FA0000000000000000000000000302000F3
:00000001FF
